:084EE00033302E3420202000A5
:10162600E4F5D975FF8075EF02751F21124BF4AFF3
:101636001F124E4043F6011248E3D2AF124CFC1281
:1016460045CA124CCB124EF8124DD0EF6010124A1A
:10165600EE123F1F3009F1C209120AA780EA1237BB
:10166600F59005B5E07002A3E060329005B6E0247F
:10167600FFF09005B5E034FFF0E07002A3E0700BD8
:101686007BFF7A4E79E0AF1F12416A30180FE49063
:1016960005B5F0A3F0A215B392151245CA1248B7C4
:1016A600EF70030217601243D4EF24FE602524FE78
:1016B600602624FC604014607414700302174324EF
:1016C600FA605124F06058241F600302175412492F
:1016D6005E807B124BB5807690054EE07005740DEA
:1016E600F080377B017A05794E900684740DF07D83
:1016F600FF1219E2802490054EE0B40D04E4F08058
:10170600117B017A05794E900684740DF07D0112E5
:1017160019E28006121A1B124EF81245CA802F9043
:1017260005B57488F0A374B8F0C21880219005310D
:10173600A3E0FAA3E0F5828A837F01800E9005314B
:10174600A3E0FAA3E0F5828A837FFF1224601248A1
:10175600B7EF60030216AC121A277B017A05799857
:0917660012488BEF700302164ECD
:10176F00C21B90059AE024FC607B147003021837AB
:10177F0024EFB40900400302188390179775F00304
:10178F00A4C58325F0C583730217B20217BC0218D4
:10179F00830218830217C30217E00218830217E8A7
:1017AF000217EED215121A15D21B021883C215D2C8
:1017BF001B0218837B017A0579989005A8EBF0A39B
:1017CF00EAF0A3E9F012226C651F60030218838010
:1017DF0000AF1F124B53021883124F0F02188312C0
:1017EF004F2E0218837B017A0579989005ABEBF0A9
:1017FF00A3EAF0A3E9F0900003122285651F70742D
:10180F0030156C9005AB04F0A3EAF0A3E9F090005B
:10181F0005122285FF900006122285FD900004120A
:10182F002285FB123CFE80477B017A057998900553
:10183F00ABEBF0A3EAF0A3E9F09000031222856569
:10184F001F70313015299005AB04F0A3EAF0A3E91E
:10185F00F0900005122285FF900006122285FD9060
:10186F000004122285FB123A7A124937124C2DAF1F
:10187F001F124BD52015030219C690059AE014606C
:10188F003624FA607414700302197224066003027E
:10189F0019C6124DE27B017A0579989005A8EBF0F5
:1018AF00A3EAF0A3E9F0900003122285F561124E2E
:1018BF00AD124ECC0219C6124DE27B017A05799812
:1018CF009005A8EBF0A3EAF0A3E9F0900003122231
:0918DF0085F561124937124ECC67
:1018E8009005B1122405000186A09005B174FF127D
:0D18F80023D2E4FBFAF9F8C31223BF40ED40
:101905000219C1124DE27B017A0579989005AEEB7B
:10191500F0A3EAF0A3E9F0900003122285FF9000FE
:1019250004122285FD900005122285FBC003900557
:10193500AEE0FBA3E0FAA3E0F99000061222859041
:0E19450005E0F0D0031239C6124937124ECC1D
:101953009005B1122405000186A09005B174FF1211
:0D19630023D2E4FBFAF9F8C31223BF40EDD4
:10197000804F124DE27B017A0579989005AEEBF02D
:10198000A3EAF0A3E9F0900003122285FF9000047F
:10199000122285FD900005122285FB122BEB1249C5
:0419A00037124ECCE0
:1019A4009005B1122405000186A09005B174FF12C0
:0D19B40023D2E4FBFAF9F8C31223BF40ED83
:1019C100124C2DD21B201B03021760121A2712453D
:0119D100CA4B
:0319D20002176099
:104D2B0075B980E4FF0FEFB414FB43B9C0E5B9309C
:054D3B00E5FB75A90372
:014D40002250
:104CB20075A41F75A5E0E4F5A675F2E77590FF757A
:094CC200D40875E10775E24222F5
:0A4EB80075A14075F80175A20322F0
:104D4100758922758E05758A5F758C5F758B4075C7
:064D51008D407588502220
:0B4E970075CA3075CBF8D2CAD2AD222C
:104BF400124D2B124CB2124EB8124D41124E971256
:0E4C04004E4D124C12124F34124DF302464820
:1033B30042042D00004203D800004203D30000C1A1
:0533C30013C112C1114D
:0A4EC200C212C213E49003D7F022DD
:104A4100E490042DF0A3F09003D8F0A3F0A3F0902C
:104A510003D3F0A3F09003CEF0A37440F0E49003ED
:034A6100D6F0226A
:064F1600124EC2024A41E6
:0D4E330075C19043E6019003D57401F02293
:104DE20043C140E5C120E5FB124F16E49003D5F024
:014DF200229E
:0A4ECC0053C1BF9003D57401F0221A
:0D4E4000AE07124E339003D2EEF0024F1673
:1049F800E49006B0F0A3F0301202FF222013FDD29B
:104A0800129003D0E4F0A37410F090041BEFF0E4CC
:044A1800A3F07F0187
:014A1C002277
:1047600030120A9003D0E07002A3E070037F0022B1
:104770009003D1E024FFF09003D0E034FFF09004E8
:104780001CE0FE04F0741D2EF582E43404F583EF82
:04479000F07F012293
:0B4EA200301207C212D213124ED622AB
:0A4ED600E5C120E5FBC2C4D2C522ED
:103F9D0090064FEBF0A3EAF0A3E9F09003D5E070A3
:103FAD0002FF22900652E0FE6005D3941040037F7D
:083FBD0000221249F8EF604EEA
:103FC500E4900654F0900652E0FF900654E0FEC3DC
:103FD5009F502490064FE0FBA3E0FAA3E0F98E8200
:103FE500758300122285FF124760EF7002FF229051
:103FF5000654E004F080CEE49003D7F0124EA29070
:0E4005000653E070032013FD9003D7E0FF2266
:034013007FFF220A
:0E35E300900685EBF0A3EAF0A3E9F0A3EDF06B
:1035F100E4FFD390042EE0940090042DE0648094C5
:103601008050012253E6FE9003D3E0FEA3E024DACA
:10361100F58274033EF583E0FF9003D3E475F00176
:10362100122393FCE5F064404C70069003D3F0A3A1
:10363100F09003CFE004F070069003CEE004F0E4D4
:10364100FE900688E0FDEEC39D5054EEC39F504F9F
:103651009003D3E0FCA3E024DAF58274033CF58304
:10366100E0FD900685E0FBA3E0FAA3E0F98E827508
:103671008300ED1222E69003D3E475F00112239347
:10368100FCE5F064404C70069003D3F0A3F0900386
:10369100CFE004F070069003CEE004F00E80A2EEBD
:1036A100C39F50299003D3E475F001122393FCE5E5
:1036B100F064404C70069003D3F0A3F09003CFE088
:1036C10004F070069003CEE004F00E80D290042E38
:1036D100E024FFF090042DE034FFF043E601900672
:0C36E10088E0FEEFC39E50028002AF069E
:0136ED0022BA
:104CE400D390042EE0940090042DE06480948040DE
:084CF400047F0180027F002211
:031A1800022A504F
:102A5000C0E0C0F0C083C082C0D075D000C000C04C
:032A600006C007A6
:102A6300C21CE5C054FE1224362B3F082B3F0A2B11
:102A7300060C2B060E2BB8102BB8122B0C222B177F
:102A8300282B172A2B0C2C2B0C2E2AF9C02AB2C266
:102A93002A9DE02A9DE200002BC3C21190041BE093
:102AA300F5C2C2C5C2C490041A74FFF0022BC590CC
:102AB300041AE0FFB4FF1290041CE0F5C2C2C5C2C1
:102AC300C490041AE4F0022BC590041CE0FEEFC38B
:102AD3009E501790041AE0FF04F0741D2FF582E452
:102AE3003404F583E0F5C2022BC5D2C49003D7E4C6
:102AF300F0C213022BC59003D774FDF0D2C5C2C434
:102B0300022BC590041A74FFF0D211C2C4C2C1D201
:102B1300C5022BC5E5C260079003D2E0B5C20E9093
:102B230003CDE4F0C2C5C2C4D2C1022BC5C2C4C224
:102B3300C1301103022BBDC2C5022BC59003CDE0EA
:102B43007020E5C2F0E0FFC39003CFE09F7480F8EC
:102B53009003CEE06480985003124A419003CDE085
:102B630004F09003CFE024FFF09003CEE034FFF0B5
:102B73009003D8E0FEA3E024DAF58274033EF583E4
:102B8300E5C2F09003D8E475F001122393FEE5F05B
:102B930064404E70069003D8F0A3F09003CDE01488
:102BA300F0700E90042EE004F0700690042DE00403
:102BB300F0D2C1800DC2C4301108C211D2C5800247
:102BC300D21C301C1053C17F43C180C2C5C2C4C2D2
:072BD300C1C21CC213C2C005
:102BDA00D007D006D000D0D0D082D083D0F0D0E0B9
:012BEA0032B8
:054F1C00E5C15420FF77
:014F2100226D
:0E454400900663EBF0A3EAF0A3E9F0A3EDF01C
:10455200E4900668F0900663E0FBA3E0FAA3E0F9BA
:10456200A3E0900652F0900667E0900653F0E4FF55
:10457200123F9DEFB4FF0D900668E0FE04F0EEC31B
:06458200940340D17E000D
:014588002210
:0B488B009006A1EBF0A3EAF0A3E9F017
:104896007E007F007D101224629006A1E0FBA3E05B
:1048A600FAA3E0F97D101235E3EF7002FF227F01D3
:0148B60022DF
:10416A009005F47422F0A3EFF0A37413F012226CFA
:10417A009005F7F09000011222859005F8F0900062
:10418A00021222859005F9F090000312228590050B
:10419A00FAF09000041222859005FBF090000512B7
:1041AA0022859005FCF09000061222859005FDF00C
:1041BA007B017A0579F4E4900667F07D0A024544AA
:104B32009006897422F0A3EFF0A37403F0A374FF2C
:104B4200F07B017A067989E4900667F07D040245DC
:014B5200441E
:104B530090068D7422F0A3EFF0A3741CF0A374FFEE
:104B6300F07B017A06798DE4900667F07D040245B7
:014B730044FD
:104BD500E4900691F0A3EFF0A3740AF0A3EFF07B45
:0F4BE500017A067991E4900667F07D0402454459
:074F080043C14053E6FE2205
:102EB700900612E0FFA3E0FCA3E0FDA3E0FBA3E084
:102EC700FAA3E0F99005EFE554F0E555A3F0900675
:062ED7001AE09005F1F085
:102EDD009005E9EFF0A3ECF0A3EDF0A3EBF0A3EA7E
:042EED00F0A3E9F075
:102EF1009005F27403F0A374E8F0E5C120E5FBD27C
:102F0100C1C2C4D2C5E4FF9006BBF030C0FDE5C02C
:102F110054FE24407003022FB424FE602424E26096
:102F21000924FE600524E2022FBCC2C5EF60030242
:102F31002FC29005E9E025E044A0F5C27F03022FEE
:102F4100C2EFB4030A9005EAE0F5C27F058072EF93
:102F5100B4050B9005EAA3E0F5C27F068063EF6438
:102F610006703E9005F1E09005EC700FE0FBA3E4E4
:102F710075F0011223A9A9F0FA8008E0FBA3E0FA99
:102F8100A3E0F912226CF5C29005F0E024FFF09065
:102F910005EFE034FFF0E07002A3E070247F0780CA
:102FA10020EFB40706D2C47F0980169006BB7405D2
:102FB100F0800E9006BB7402F080069006BB74018F
:102FC100F0EFB40904C2C080369006BBE0FE64068F
:102FD1006012EEB402169005F274FFF5F01223931D
:102FE10045F06008D2C5E49006BBF0FF9006BBE057
:102FF1006008C2C5D2C4C2C08005C2C0022F0CE5A0
:04300100C120E5FB0A
:0130050022A8
:103006009005FEEFF0A3ECF0A3EDF0A3EBF0A3EA3E
:04301600F0A3E9F04A
:10301A009006067403F0A374E8F0E5C120E5FBD23C
:10302A00C1C2C4D2C5E4FF9006BBF030C0FDE5C002
:10303A0054FE24C870030230F724AE607A24CA70A2
:10304A00030230FF24FE603824E2600924FE600592
:10305A0024E2023107C2C5EF700F9005FEE025E0B9
:10306A0044A0F5C27F0302310DEF6401600302310F
:10307A000D9005FEE025E044A1F5C27F0402310D62
:10308A00EFB4030A9005FFE0F5C27F058075EFB43F
:10309A00050B9005FFA3E0F5C27F068066EFB40634
:1030AA0006D2C57F01805CEFB404047F028054908D
:1030BA0006BB7405F0804C900601E0FBA3E475F0B2
:1030CA00011223A9A9F0FAE5C21222D4900605E05A
:1030DA0024FFF0900604E034FFF0E07002A3E070F1
:1030EA00087F09C2C1D2C4801A7F0280169006BB2B
:1030FA007406F0800E9006BB7402F080069006BB40
:10310A007401F0EFB40904C2C080369006BBE0FE39
:10311A0064066012EEB4021690060674FFF5F01209
:10312A00239345F06008D2C5E49006BBF0FF9006F1
:10313A00BBE06008C2C5D2C4C2C08005C2C00230AA
:06314A0035E5C120E5FBA4
:01315000225C
:1036EE00900612EFF0900615EBF0A3EAF0A3E9F0C6
:0836FE00900613ECF0A3EDF0BF
:10370600755600543FF557543F605CC37440955757
:10371600FFE49556FE900618E0FCA3E0FDC39FEC7F
:103726009E50068C548D5580048E548F55122EB79C
:103736009006BBE060037F0222900614E02555F058
:10374600900613E03554F090061AE0700B900616BA
:10375600E5548555F0122393C3900619E09555F06C
:10376600900618E09554F0900618E0F554A3E0F59D
:1037760055D3E5559400E55494004070E5559440C2
:10378600E55494005013122EB79006BBE060037FF9
:103796000222E4F554F55580D8900612E0FFA3E026
:1037A600FCA3E0FDA3E0FBA3E0FAA3E0F99005EF9C
:1037B600E4F07440122ED39006BBE060037F022231
:1037C60074C02555F55574FF3554F554900614E02C
:1037D6002440F0900613E03400F090061AE0709151
:0E37E60090061675F0401223930237777F008D
:0137F40022B2
:104D1400900604E4F0A304F01230069006BBE060B1
:074D2400037F01227F002242
:104C7E009006BAEBF07B017A0679BA900618E4F04A
:0A4C8E00A304F0E4A3F01236EE22B6
:104AAA00C00790063CE0FFA3E0900604CFF0A3EF16
:104ABA00F0D0071230069006BBE060037F01227F28
:024ACA000022C8
:104C9800C007900644E0FFA3E0900618CFF0A3EF0A
:0A4CA800F0E4A3F0D0071236EE226C
:104B7400A2AFE433FCC2AF758F0175B7A575B7F169
:104B84008F828E83EDF0E4F58FAF04EF24FF92AFB4
:014B940022FE
:104B9500A2AFE433FDC2AF758F0375B7A575B7F145
:0F4BA5008F828E83E4F0F58FAF05EF24FF92AF80
:014BB40022DE
:10442500900695EEF0A3EFF0A3ECF0A3EDF0EB4AC8
:104435006039900695E0FEA3E0FFA3E0FCA3E0F55C
:10444500828C83E0FD124B74EB1B70011A90069869
:10445500E004F07006900697E004F0900696E004FC
:0C446500F070CB900695E004F080C322BC
:084EE800E4900051F0A3F02258
:1049AC00900051E0FEA3E0FF124B95900051E0FE09
:1049BC00A3E0FF7C007D537B007A02124425E49037
:0649CC000051F0A3F022EF
:0A3D9100A905900669EEF0A3EFF01B
:103D9B00EE54FEFE900051E0FCA3E0FD7002EE6CD1
:103DAB006057ED4C60031249AC900669E0FEEE548F
:103DBB00FEFE7F00900051F0A3EFF090066BEEF04B
:103DCB00A3EFF0A37400F0A37453F07E0290066B84
:103DDB00E475F0011223A985F082F583E493FD903D
:103DEB00066DE475F0011223A985F082F583EDF0E1
:103DFB00EF1F70011EEF4E70D4900669E0FCA3E03C
:103E0B00FDEC5401FC74532DF58274003CF583E9F1
:013E1B00F0B6
:013E1C002283
:1044B800900655EEF0A3EFF0A3EBF0A3EAF0A3E922
:1044C800F090065A74FFF5F01223A945F060269083
:1044D8000655E475F0011223A9AFF0FE900657E0E7
:1044E800FBA3E475F0011223A9A9F0FA12226CFDCE
:0644F800123D9180CC2270
:1033C8000212000048048C023602340237023548E3
:1033D800048402320233013000304804940230027F
:1033E80031013100314C04BC013201330134003267
:1033F800003300344C04C80137013601350037006A
:0334080036003556
:104DBD007F008F178F147F1B8F188F157F368F19DC
:034DCD008F16221C
:06460A007B017D047C0031
:1046100090067BEBF0A3EAF0A3E9F0A3ECF0A3EDA6
:10462000F090067E74FFF5F01223A945F060189013
:10463000067BE0FBA3E475F0021223A9A9F0FAE4DB
:08464000FDFC123BD880DA22D8
:104648007E007F207D007B017A04799C122462120F
:104658004DBD7A04798C12460A7A04798412460A86
:104668007B017A04799412460C7B017A0479BC7D2B
:09467800067C001246100237F521
:0A3BCE007B0135F0FAE0FCA3E0FDF6
:103BD8009006B2ECF0A3EDF0C2AD12226C14602F87
:103BE80014605424027075900001122285A814F202
:103BF8009006B2E0FEA3E0FFE804F8EEF208EFF268
:103C0800E5142403F514641B7052751400804D905C
:103C18000001122285A815F29006B2E0FEA3E0FF8B
:103C2800E804F8EEF208EFF2E5152403F51564361A
:103C3800702A75151B8025900001122285A816F29E
:103C48009006B2E0FEA3E0FFE804F8EEF208EFF217
:103C5800E5162403F516B45103751636D2ADD21DF8
:013C68002239
:0E3EA00090065CEFF0A3ECF0A3EDF0A3EBF0C6
:103EAE00D394665018E0FD75F080A4FBED25E0FE7E
:103EBE00E42BFFEE35F0900661F0A3EFF090065C78
:103ECE00E075F002A4248CF9740435F0FA7B01A39A
:103EDE00123BD390065FE0601390065CE075F00233
:103EEE00A42484F97404900661123BD0900660E01D
:103EFE00601E90065CE075F002A42494F9740435FB
:103F0E00F0FA7B01900660E07D0025E0FC123BD8C4
:013F1E002280
:053B2D009006B4EFF06A
:103B3200ED75F00AA42495F582E43402F583E0FEE3
:103B42009006B5F0EF75F005A42458F582E434032D
:103B5200F583E0FB3395E0FAEEFF7E00EB2FFFEEFC
:103B62003AFED3EF947FEE6480948040089006B5CD
:103B7200747FF08014C3EE648094805007E4900652
:103B8200B5F080059006B5EFF09006B4E0FF24088A
:103B9200F876F0EF75F005A42456F582E43403F5C7
:103BA20083E0FFED75F00AA42496F582E43402F571
:103BB20083E0FD7C001238FC900660EFF09006B4C2
:0C3BC200E0FFA3E0FB74FFFDFC023EA04E
:10458900EF25E025E0249CF582E43404F5837401E9
:10459900F00513E513AA127002051214FBEF25E0CA
:1045A90025E0249EF582E43404F583EAF0A3EBF0D8
:1045B900EF25E025E0249DF582E43404F583EDF050
:0145C90022CF
:1049D200EF25E025E0249EF582E43404F583E0FA35
:1049E200A3E0FBC39511EA9510500A8A108B118F30
:0649F2000DAF058F0F223E
:100AA700E49004D4F09004D4E0FFC394045029EFF9
:100AB70075F008A424D9F582E43404F583740FF0A3
:100AC700EF75F008A424DAF582E43404F583E4F042
:100AD7009004D4E004F080CDE49004D5F09004D5E0
:0A0AE700E0FFC39410400302162341
:100AF100EF75F00AA42493F582E43402F583E090C3
:080B010004FAF0700302161A59
:100B0900A37401F09004D5E075F00AA42494F58249
:100B1900E43402F583E09004FCF0E49004D4F0900E
:100B290004D4E0FFC3940840030215BEEF6003B488
:100B3900040DE4F50FF50EF50D74FFF510F511EF41
:100B490075F005A42440F582E43403F583E0FF90B1
:100B590004D5E0FEEF6E60030212379004D4E0FF83
:100B690075F005A42441F582E43403F583E07003AC
:100B7900020DA09004FAE064016035EF25E025E05C
:100B8900249CF582E43404F583E070030212379063
:100B990004D4E025E025E0249DF582E43404F583BE
:100BA900E0FE9004FCE0FDEE6D6003021237801C4C
:100BB900E50E60030212379004D4E0FF25E025E03A
:100BC900249CF582E43404F583E0600B9004FBE097
:100BD900FD1249D2021237750E019005B7E0FF9058
:100BE90004FBE0FEEF4E9005B7F09004D4E0FF90CF
:100BF90004FCE0FD1245899004D4E0FFC39404404D
:100C090003020D90A3E075F00AA42495F582E4345B
:100C190002F583E0FD7C00EF75F005A42444F5821C
:100C2900E43403F583E0FF3395E0FEEF2DFFEC3E5E
:100C3900FE9004F7F0A3EFF0D3947FEE64809480E4
:100C4900400B9004F7E4F0A3747FF0800FC3900485
:100C5900F7E0648094805004E4F0A3F09004F7A3D3
:100C6900E0547FA3F0E49004D6F09004D6E0FFC3EB
:100C790094044003021237EF75F008A424DAF582D0
:100C8900E43404F583E06003020D239004D6E07593
:100C9900F008A424DAF582E43404F5837490F09022
:100CA90004F9E0FEEF75F008A424DCF582E43404CD
:100CB900F583EEF09004D4E075F005A42442F582A2
:100CC900E43403F583E0FF9004D5E075F00AA42429
:100CD90096F582E43402F583E0FD7C001238FC903D
:100CE90004D6E0FE75F008A424DDF582E43404F5A9
:100CF90083EFF0EE75F008A424DAF582E43404F504
:100D090083C083C082E0FF9004D4E0FE7408A80683
:100D1900088002C313D8FC4F80599004D6E0FF75B0
:100D2900F008A424DAF582E43404F583E0FE54F0F3
:100D39006490704AEF75F008A424DCF582E4340469
:100D4900F583E0FF9004F9E0FDEFB505319004D695
:100D5900E075F008A424DAF582E43404F583C0834D
:100D6900C0829004D4E0FF7408A807088002C31366
:100D7900D8FC4ED082D083F09004D67404F090044D
:100D8900D6E004F0020C739004D4E024FCFFA3E045
:100D9900FD123B2D0212379004FAE0FC9005B7B41E
:100DA900030CE0FE9004FBE0F4FDEE5D8009E0FF3A
:100DB9009004FBE0FEEF4E9005B7F09004D4E0FFFD
:100DC900C3940440030210E4EC64036003020F5C63
:100DD900A3E075F00AA42495F582E43402F583E0D2
:100DE900FD7C00EF75F005A42444F582E43403F595
:100DF90083E0FF3395E0FEEF2DFFEC3EFE9004F714
:100E0900F0A3EFF0D3947FEE64809480400B9004BC
:100E1900F7E4F0A3747FF0800FC39004F7E06480D7
:100E290094805004E4F0A3F09004F7A3E0547FA366
:100E3900F0E49004D6F09004D6E0FFC39404400394
:100E4900021237EF75F008A424DAF582E43404F5C8
:100E590083E06003020EEF9004D6E075F008A42445
:100E6900DAF582E43404F5837480F09004F9E0FE45
:100E7900EF75F008A424DCF582E43404F583EEF080
:100E89009004D4E075F005A42442F582E43403F516
:100E990083E0FF9004D5E075F00AA42496F582E476
:100EA9003402F583E0FD7C001238FC9004D6E0FEA4
:100EB90075F008A424DDF582E43404F583EFF0EE3F
:100EC90075F008A424DAF582E43404F583C083C0FC
:100ED90082E0FF9004D4E0FE7408A806088002C3EB
:100EE90013D8FC4F80599004D6E0FF75F008A4246C
:100EF900DAF582E43404F583E0FE54F06480704A44
:100F0900EF75F008A424DCF582E43404F583E0FFEE
:100F19009004F9E0FDEFB505319004D6E075F008CD
:100F2900A424DAF582E43404F583C083C0829004F2
:100F3900D4E0FF7408A807088002C313D8FC4ED078
:100F490082D083F09004D67404F09004D6E004F0C3
:100F5900020E3F9004D5E075F00AA42495F582E4C9
:100F69003402F583E0FF7E009004D4E075F005A417
:100F79002444F582E43403F583E0FD3395E0FCED88
:100F89002FFFEE3CFE9004F7F0A3EFF0D3947FEE31
:100F990064809480400B9004F7E4F0A3747FF080A0
:100FA9000FC39004F7E0648094805004E4F0A3F048
:100FB9009004F7A3E0547FA3F0E49004D6F09004E2
:100FC900D6E0FFC394044003021237EF75F008A47A
:100FD90024DAF582E43404F583E0600302107790A3
:100FE90004D6E075F008A424DAF582E43404F58324
:100FF9007490F09004F9E0FEEF75F008A424DCF594
:1010090082E43404F583EEF09004D4E075F005A48D
:101019002442F582E43403F583E0FF9004D5E075BA
:10102900F00AA42496F582E43402F583E0FD7C00FD
:101039001238FC9004D6E0FE75F008A424DDF58290
:10104900E43404F583EFF0EE75F008A424DAF582B0
:10105900E43404F583C083C082E0FF9004D4E0FE49
:101069007408A806088002C313D8FC4F805990045D
:10107900D6E0FF75F008A424DAF582E43404F58398
:10108900E0FE54F06490704AEF75F008A424DCF592
:1010990082E43404F583E0FF9004F9E0FDEFB5053F
:1010A900319004D6E075F008A424DAF582E434041A
:1010B900F583C083C0829004D4E0FF7408A80708B0
:1010C9008002C313D8FC4ED082D083F09004D6742A
:0B10D90004F09004D6E004F0020FC702
:1010E400E4900503F0A3F09004FAE0B4030AE4905A
:1010F40004FDF0A3F00211D674FF9004FDF0A3F0F8
:10110400900503E4F0A374F0F09004D4E075F005C6
:10111400A42442F582E43403F583E0FF9004D5E08F
:1011240075F00AA42496F582E43402F583E0FD7C8C
:10113400001238FCEF25E09004FFF0A3E4F09004E3
:10114400D4E075F005A42444F582E43403F583E087
:10115400FF3395E0FE9004D5E075F00AA42495F5DC
:1011640082E43402F583E02FFFE43EFE900506F0AE
:10117400A3EFF0D3947FEE64809480400B90050637
:10118400E4F0A3747FF0800FC3900506E0648094BC
:10119400805004E4F0A3F0900506E0FCA3E0FD54C5
:1011A4007F25E0900501F0A3E4F0D3ED9466EC64B0
:1011B400809480501D900506E0FEA3E07807C333B9
:1011C400CE33CED8F9FF900502E02FF0900501E070
:1011D4003EF09004D4E024FC900505F0900503A3B0
:1011E400E0FFA3E0FE2408F8A6079004FAE06402F6
:1011F4006010EE75F002A4248CF974049004FD12BE
:101204003BCE9004FAE064036029900505E075F094
:1012140002A42484F97404900501123BCE900505C0
:10122400E075F002A42494F9740435F0FA9004FFF4
:03123400123BD397
:101237009004FBE025E0F09004D4E0FF640360082D
:10124700EF640760030215B59004FAE064017003C8
:1012570002140DE50F700302140D9005B7E0FFE5CA
:101267000FF4FEEF5EF0E50D25E025E0249CF58206
:10127700E43404F583E4F0E50DC39404400302135A
:10128700FA9004D5E075F00AA42495F582E43402B7
:10129700F583E0FF7E00E50D75F005A42444F58293
:1012A700E43403F583E0FD3395E0FCED2FFFEE3CDE
:1012B700FE9004F7F0A3EFF0D3947FEE6480948060
:1012C700400B9004F7E4F0A3747FF0800FC3900401
:1012D700F7E0648094805004E4F0A3F09004F7A34F
:1012E700E0547FA3F0E49004D6F09004D6E0FFC367
:1012F700940440030215B5EF75F008A424DAF582CB
:10130700E43404F583E060030213989004D6E07593
:10131700F008A424DAF582E43404F5837480F090AD
:1013270004F9E0FEEF75F008A424DCF582E4340448
:10133700F583EEF0E50D75F005A42442F582E4345B
:1013470003F583E0FF9004D5E075F00AA42496F531
:1013570082E43402F583E0FD7C001238FC9004D669
:10136700E0FE75F008A424DDF582E43404F583EF8C
:10137700F0EE75F008A424DAF582E43404F583E08E
:10138700FFAE0D7408A806088002C313D8FC4F806F
:10139700529004D6E0FF75F008A424DAF582E4340D
:1013A70004F583E0FE54F06480703FEF75F008A405
:1013B70024DCF582E43404F583E0FF9004F9E0FDD2
:1013C700EFB505269004D6E075F008A424DAF58277
:1013D700E43404F583AF0D7408A807088002C3132B
:1013E700D8FC4EF09004D67404F09004D6E004F0D4
:1013F7000212F1E50D24FCFFE4900660F0FBFDFC12
:10140700123EA00215B5E50E60030215B5E50F7093
:10141700030215B59005B7E0450FF09004FCE0FD19
:10142700AF0D124589E50DC3940440030215A8903A
:1014370004D5E075F00AA42495F582E43402F58317
:10144700E0FF7E00E50D75F005A42444F582E43441
:1014570003F583E0FD3395E0FCED2FFFEE3CFE90B6
:1014670004F7F0A3EFF0D3947FEE64809480400BF1
:101477009004F7E4F0A3747FF0800FC39004F7E0C3
:10148700648094805004E4F0A3F09004F7A3E05440
:101497007FA3F0E49004D6F09004D6E0FFC3940451
:1014A70040030215B5EF75F008A424DAF582E43499
:1014B70004F583E060030215469004D6E075F00852
:1014C700A424DAF582E43404F5837490F09004F9E7
:1014D700E0FEEF75F008A424DCF582E43404F5831C
:1014E700EEF0E50D75F005A42442F582E43403F52A
:1014F70083E0FF9004D5E075F00AA42496F582E412
:101507003402F583E0FD7C001238FC9004D6E0FE3F
:1015170075F008A424DDF582E43404F583EFF0EEDA
:1015270075F008A424DAF582E43404F583E0FFAE0D
:101537000D7408A806088002C313D8FC4F80529088
:1015470004D6E0FF75F008A424DAF582E43404F544
:1015570083E0FE54F06490703FEF75F008A424DC3C
:10156700F582E43404F583E0FF9004F9E0FDEFB57C
:1015770005269004D6E075F008A424DAF582E43451
:1015870004F583AF0D7408A807088002C313D8FCBD
:101597004EF09004D67404F09004D6E004F00214E0
:1015A7009FE50D24FCFF9004D5E0FD123B2D900430
:1015B700D4E004F0020B28E49004D6F09004D6E0BF
:1015C700FF75F008A424DAF582E43404F583E060BB
:1015D7002FEF75F008A424D7F9740435F0FA7B01CE
:1015E7007D08124E8B9004D6E075F008A424DAF536
:1015F70082E43404F583E4F09004D6E004F080BC80
:101607009004D5E075F00AA42493F582E43402F53A
:0316170083E4F079
:0C161A009004D5E004F0020AE40245CA86
:1037F500201D030238FBC21DE514B5170EE515B5EE
:0B3805001809E516651970030238FB76
:10381000C283E516B519089006A474F0F08020A8BC
:1038200019E29006A4F0E804F8E2FF08E2A3CFF062
:10383000A3EFF0E5192403F519B45103751936E423
:10384000FF124EF09006A4E0FF124EF09006A5E0A5
:10385000FF124EF09006A5A3E0FF124EF0E515B55D
:1038600018089006A474F0F08020A818E29006A42E
:10387000F0E804F8E2FF08E2A3CFF0A3EFF0E518C8
:103880002403F518B4360375181BE4FF124EF090AC
:1038900006A4E0FF124EF09006A5E0FF124EF09055
:1038A00006A5A3E0FF124EF0E514B517089006A494
:1038B00074F0F08020A817E29006A4F0E804F8E283
:1038C000FF08E2A3CFF0A3EFF0E5172403F517B448
:1038D0001B03751700E4FF124EF09006A4E0FF12E0
:1038E0004EF09006A5E0FF124EF09006A5A3E0FF73
:0838F000124EF0124F22D283A8
:0438F8000237FD2274
:104ACC0074082FF8E6601A16E67016EF75F002A45B
:104ADC00248CF9740435F0FA7B017D007C80123B48
:024AEC00D822CE
:031A12000242DAB3
:1042DA00C0E0C0F0C083C082C0D075D000C000C0AA
:0D42EA0001C002C003C004C005C006C0072B
:1042F700C2CF9006BCE4F09006BCE0FFC394045024
:0C4307000B124ACC9006BCE004F080EBE6
:10431300D007D006D005D004D003D002D001D000FE
:0B432300D0D0D082D083D0F0D0E032A8
:104E150000FF0100010000FFFF0000010001FF008D
:07340B004205B50000C118E5
:053E1D00900699EFF092
:103E2200E54C2401FFE4354BFAA907A37401F0A382
:103E3200EAF0A3E9F090069AE0FBA3E0FAA3E0F926
:103E420074019005CC6B7008E965827003EA6583A2
:103E5200700D90069A04F0A37405F0A374B8F09064
:103E6200069AE0FBA3E0FAA3E0F9E54D854E8385CF
:103E72004F826B7008E965827003EA6583601E9069
:103E82000699E0854C82854B83F090069AA3E0FA6E
:0D3E9200A3E0AE028E4BF54C900699E0F0D7
:013E9F002200
:074D57009006A7E0FFAD4943
:0E4D5E00EB5F6009ED5B6005AF03123E1D22A6
:0D4E4D0075BC4475E8C075BA1F75D1082208
:1043D40053E6EFE54D854E83854F826401700AE50F
:1043E4004C65827004E54B65837003FF802FAB4DF1
:1043F400054FE54FAA4E7002054E14F912226CFFC8
:1044040074019005CC6B700AE54F65827004E54E2B
:1044140065837009754D01754E05754FB843E610F7
:014424002275
:1048B70053E6EFE54D854E83854F826401700AE527
:1048C7004C65827004E54B65837003FF800AAB4D2E
:0B48D700AA4EA94F12226CFF43E6100E
:0148E20022B3
:104A6400EFD394B840047E108016EFD394784004BA
:104A74007E04800CEFD3945040047E018002E4FE57
:024A8400AF067B
:014A8600220D
:031A24000231513B
:10315100C0E0C0F0C083C082C0D075D000C001C043
:0F31610002C003C005C006C00720DF03023216FC
:103170009006A8E5BEF0D2ECA217B3921730170D57
:1031800075BB04E0FF124A648F4902321475BB0319
:103190009006A8E0FF124A64EF25E04249E5496540
:1031A000536012E54965539006A7F0543F600375DC
:1031B0005103854953E551605B1551E5517055E563
:1031C0005265499006A7F09005B5E07002A3E06053
:1031D00006E5497002D2187B01124D577B02124D51
:1031E000579006A7E0FF7B04AD49124D5E9006A7FD
:1031F000E0FF7B08AD49124D5E9006A7E0FF7B1013
:10320000AD49124D5E9006A7E0FF7B20AD49124DFF
:063210005E854952C2DF99
:0632160020D80330D95856
:10321C009006A7E590F0C2D9C2D8E0FD65505403E2
:10322C006046E55075F004A47E00540CFFED540389
:10323C00FDEF4D2415F582EE344EF583E493FF90AB
:10324C0006A8F0A3E54AF0EF254AF54AE0654A30B6
:10325C00E1109006A8E0B401047F0980027F0A12F5
:08326C003E1D9006A7E0F5509D
:10327400D007D006D005D003D002D001D0D0D08260
:07328400D083D0F0D0E0324E
:0C4E670075DA3175DB3175D989D2DE2295
:104C1200124E677B017A0579B88B4D8A4E894F8A8D
:0B4C22004B894CE49005B7F00245CA36
:064F2200E5A120E7FB22DF
:084EF000E5A120E7FB8FA322DE
:1045CA007D017C00E4FB90054EE0FFEBC39F500A9F
:1045DA00ED25E0FDEC33FC0B80EC301504EC444097
:1045EA00FCC2AFD2839005B7E0F4FF124EF0ECF4B0
:0F45FA00FF124EF0EDF4FF124EF0124F22D2AF2F
:01460900228E
:103412006054042F00010204081000000304180085
:10342200000000001F00000000001804030000005C
:103432000010080402010000040A0A111100000130
:103442000102021C00001C0202010100001010080F
:1034520008070000070808101000001818001818C4
:083462000000181803181800FF
:064F28001247948FA02245
:0D4E25007FC87E00EF1F70011EEF4E70F77A
:014E3200225D
:104DF3007F38124D817F06124D817D0EE4FF024EF6
:014E0300733B
:104D81009006BDEFF0124D6CEF20E7F99006BDE003
:044D9100FF024D953B
:104D6C0075A0FFC296D295D2977F14DFFEAFA0122A
:044D7C004794C297FF
:014D80002210
:054F40007F01024D811C
:104D9500124F28124E25C296C295D297124E25C2A1
:044DA50097024E25FE
:104E0400124F28C295D297D296124E25C297024EBF
:014E14002578
:0C4E7300900483E05FF04DFFF0024D81E1
:0F4A8700A3E475F0011223A9A9F0FA12226CFF23
:104A96009006BEEFF0124D6CEF20E7F99006BEE0EF
:044AA600FF024E04B9
:104A1D009006AAEBF0A3EAF0A3E9F09006AAE0FB5A
:104A2D00A3E0FAA3E0F912226C60089006AA124ADC
:044A3D008780E82264
:1046F30090066FEBF0A3EAF0A3E9F0124F40E4FD5C
:10470300FF124E7F90066FE0FBA3E0FAA3E0F912DD
:104713004A1DE4FD7F01124E7F900672E0FBA3E089
:07472300FAA3E0F9024A1DB0
:0C4E7F00EF75F040A42D2480FF024D814F
:08428400900675EFF0A3EDF0C8
:10428C00E075F008A42440FF124D81900675E054AF
:10429C007F75F007A4242FF9740435F0FA90067892
:1042AC007401F0A3EAF0A3E9F0900676E0900675AD
:1042BC00F09006777407F0900677E0FF14F0EF604B
:0E42CC0008A3E0FB124A8780EEE4FF024A9648
:10479400E4F55DF55EF55CAE5C7480A80608800205
:1047A400C313D8FCF55D5F600FAE5C7401A8060806
:1047B4008002C333D8FC425E055CE55CB408D8AF24
:0147C4005E96
:0147C50022D1
:10346A00C10EC10F4E025500020002000200020006
:10347A00010001000241033F004A0289603020181E
:0E348A00100C080604034102530041025400D6
:031A1500D20F22CB
:034F4500C20F2276
:104CCB007E007FA07D007B017A027993122462E43F
:094CDB009005B7F0C20DC20A22D7
:091A1B00124CCB124648D20922FC
:084EF800E4F55FF560C20E2233
:0C4E8B00300F08E4900667F01245442246
:1038FC00EF14B4090040030239C390391475F00376
:10390C00A4C58325F0C583730239680239320239A4
:10391C005F02392F02397302394D0239370239846B
:10392C000239A20239BE7D500239C374C12DFD7417
:10393C00FF3CC3648094805002E4FDED25E0FD80E3
:10394C007174C12DFD74FF3CC3648094805041E4BC
:10395C00FD803DC374809DFDE49C8001ECA2E713C7
:10396C00ED13243CFD8050D3ED943FEC64809480A7
:10397C004004747F9DFD8018C374809DFDE49CFC05
:10398C0074C12DFD74FF3CC3648094805002E4FD2F
:10399C00ED25E0FD8021C374809DFDE49CFC74C189
:1039AC002DFD74FF3CC3648094805002E4FDED2532
:0A39BC00E0FDC374809DFDAF0522FD
:104C2D00E49006BFF09006BFE0FFC39404500B1252
:0A4C3D0044FE9006BFE004F080EB97
:014C4700224A
:0244FE00AD0708
:10450000900648740FF07408A807088002C313D8F7
:10451000FC44B0900649F090064B741FF0ED75F026
:1045200005A42443F582E43403F583E090064CF0BF
:10453000300F107B017A067946E4900667F07D081B
:03454000124544DD
:014543002255
:0C401600F583E0FEC4540FFFEE540FFDD4
:10402200AB05AA0774892BF582E43402F583E0FD1F
:104032003395E0FCE56024FFFFE55F34FFFE1223C9
:054042005DED4C70462D
:1040470074892BF582E43402F583E0FD3395E0FCB7
:10405700E56024FFFFE55F34FFFE1223089006B6F4
:10406700EEF0A3EFF0E004F070069006B6E004F07F
:104077000AEAFD7C009006B6E0FEA3E0FF122308E3
:06408700ED4C7002D32293
:02408D00C3224C
:102D5D00E49006C0F09006C0E0FFC3940640030265
:102D6D002EB6EF75F005A42468F582E43403F583DF
:102D7D00E064106003022EAD9006C0E075F005A46E
:102D8D002469F582E4340312401650319006C0E0F8
:102D9D0075F002A424BCF9740435F0FA7B0174FFBC
:102DAD00FDFC123BD8900253E0FF9006C0E0FE748C
:102DBD0001A806088002C333D8FC4F804B9006C093
:102DCD00E0FD74017E00A805088005C333CE33CE27
:102DDD00D8F9FF900253E0FBEF5B6030ED75F00228
:102DED00A424BCF9740435F0FA7B01E4FDFC123B1C
:102DFD00D8900253E0FF9006C0E0FE7401A80608CB
:102E0D008002C333D8FCF45F900253F09006C0E00B
:102E1D0075F005A4246AF582E4340312401650318E
:102E2D009006C0E075F002A424C8F9740435F0FAD8
:102E3D007B0174FFFDFC123BD8900254E0FF90061D
:102E4D00C0E0FE7401A806088002C333D8FC4F8091
:102E5D004B9006C0E0FD74017E00A805088005C3F7
:102E6D0033CE33CED8F9FF900254E0FBEF5B6030E8
:102E7D00ED75F002A424C8F9740435F0FA7B01E471
:102E8D00FDFC123BD8900254E0FF9006C0E0FE74AA
:102E9D0001A806088002C333D8FCF45F900254F0F9
:092EAD009006C0E004F0022D6261
:012EB60022F9
:0E27A3009005CCEFF0A3ECF0A3EDF0A3EBF06B
:1027B1009005D174B0F0A374E0F09005D5740FF0DA
:1027C100E49005D0F09005D0E0FFC39404505DEF94
:1027D10075F005A42440F582E43403F583E0FF900D
:1027E10005CFE0FEEF6E703C9005CCE0701C9005CB
:1027F100D2E0FF9005D0E0FE7408A806088002C36D
:1028010013D8FC4F9005D2F0801A9005D1E0FF90CB
:1028110005D0E0FE7408A806088002C313D8FC5F47
:102821009005D1F09005D0E004F08099E49005D0B6
:10283100F09005D0E0FFC3940640030228E9EF754C
:10284100F005A42469F582E43403F583E0FF9005E3
:10285100CCE0FEEF6E70379005D0E0FF75F005A477
:102861002468F582E43403F583E0FE9005CFE0FDB2
:10287100EEB5051AEF75F002A424BCF9740435F025
:10288100FA7B019005CDE0FCA3E0FD123BD8900559
:10289100D0E0FF75F005A4246AF582E43403F583E2
:1028A100E0FE9005CCE0FDEE6D7034EF75F005A40F
:1028B1002468F582E43403F583E0FF9005CFE0FE60
:1028C100EFB5061BA3E075F002A424C8F974043522
:1028D100F0FA7B019005CDE0FCA3E0FD123BD8901E
:1028E10005D0E004F00228329005D1E0FF540F60DA
:1028F100299005D6EFF09005CCE09005D8F0900531
:10290100CDA3E09005D9F0300F107B017A0579D382
:10291100E4900667F07D081245449005D2E0FF542B
:102921000F60389005D6EFF09005CDE0FCA3E0FDF7
:10293100AE047802CEC313CE13D8F9547F9005D8D4
:10294100F0ECC313547FA3F0300F107B017A0579AB
:10295100D3E4900667F07D081245449005CCE0640D
:10296100426003022A4F9005CFE090033FF0A20A94
:10297100920DC39005CDE094804003022A4DC20A16
:06298100200D03022A4FA5
:062987009005DB7403F073
:10298D009005DC7403F09005DCE0FFC36480948057
:10299D004058EF3395E0FEEF25E0FFEE33FE900358
:1029AD003FE0FD75F00AA42496F582E43402F58328
:1029BD00E5822FF582E5833EF583E4F074372FF53C
:1029CD008274033EF583E0FCED75F00AA42495F5C1
:1029DD0082E43402F583E5822FF582E5833EF583AB
:1029ED00ECF09005DCE014F0809C90033FE0FD7569
:1029FD00F00AA42493F582E43402F5837403F09075
:102A0D0005DBE0FF3395E0FEEF25E0FFEE33FE74CE
:102A1D00372FF58274033EF583E0FFED75F00AA4C0
:0E2A2D002494F582E43402F583EFF0120AA738
:102A3B009005DBE014F0E0C364809480400302292E
:022A4B008D22DA
:022A4D00D20AAB
:012A4F002264
:1024AE00C21E90061D740FF0EF122436258980246B
:1024BE00DC9026EDA026FFB02717C026CCE02766BD
:1024CE00F82736FA275AFB274EFC0000278C90027D
:0724DE006DE0700302258987
:1024E5009006237402F0900264E075F00AA4FDAC36
:1024F500F02495F974023CFA7B01900623E0FF3342
:1025050095E0FEEF25E0FFEE33FEE92FF9EA3EFA0E
:10251500C002C00174972DF974023CFAE92FF9EA5B
:102525003EA801FC7D01D001D0027E007F0212226F
:1025350046900623E014F0E0C36480948050A79091
:10254500026CE0FF900264E0FE75F00AA42495F5A4
:1025550082E43402F583EFF090026DE0FDEE75F054
:102565000AA42496F582E43402F583EDF0EE75F0C5
:102575000AA42493F582E43402F5837401F0D209A8
:04258500EE0226BA82
:10258900300A629006237402F0900623E0FFC364C8
:102599008094804044EF3395E0FEEF25E0FFEE3371
:1025A900FE74372FF58274033EF583E0FD74392FED
:1025B900F58274033EF583EDF074382FF5827403C8
:1025C9003EF583E0FD743A2FF58274033EF583ED01
:1025D900F0900623E014F080B090026CE09003378D
:1025E900F0E4A3F022E4900623F0900623E0FFC371
:1025F9006480948440030226B1EF3395E0FEEF2511
:10260900E0FFEE33FE900264E075F00AA42495F52C
:1026190082E43402F583E5822FF582E5833EF58372
:10262900E0FF90026CE0FEEF6E7074900623E0C349
:10263900648094835053900264E075F00AA4FDAC61
:10264900F02497F974023CFA7B01900623E0FF33EA
:1026590095E0FEEF25E0FFEE33FEE92FF9EA3EFAB9
:10266900C002C00174952DF974023CFAE92FF9EA08
:102679003EA801FC7D01D001D0027E007F0212221A
:1026890046900623E004F080A2900264E075F00A07
:10269900A42493F582E43402F5837403F0D20990FB
:1026A9000623E004F00225F390026CE0FF90026437
:1026B900E075F00AA42494F582E43402F583EFF07E
:0326C90002278C59
:1026CC0090026CE075F004A4FDA3E025E0FEE42D7F
:1026DC00FFEE35F0FEAD07FC900264E0FBE4FF80FA
:1026EC002590026DE07D0025E0FC900264E0FB7F0C
:1026FC0001801390026CE02402FFA3E07D0025E032
:10270C00FC900264E0FB1227A3807590026CE0FF42
:10271C00C3941E506B90061E74C0F0900264E0903F
:10272C00061FF0A3EFF0D21E8056D20EE490025397
:10273C00F0A3F090061E74FAF0D21EE4F55FF5607B
:10274C00803E90061E74FCF0D21EC20E80329006A3
:10275C001E74FBF0D21ED20E8026300E2390061E65
:10276C0074F8F0D21E0560E560AE5F7002055F1470
:10277C00B4000AEEB40306755F00756001122D5D9E
:10278C00301E13300F107B017A06791BE49006671C
:06279C00F07D0812454427
:0127A2002214
:1040FE00AE07EF7008900265F0A3F08057EE54F013
:10410E00900263F0EE540FA3F0EEC394F0402690AD
:10411E000263EEF0B4F00BE4900269F0900267F0E7
:10412E00A3F0EEC394F85005E490026AF090026496
:10413E0074FFF0801F90026AEEF0C4540F25E02445
:10414E0045F582E43402F583E0FFA3E0900265CFEB
:0C415E00F0A3EFF0E4900267F0A3F02261
:103F1F009006C1EFF030E72AE0FFB4FF0122EF6413
:103F2F00F8600EEF64FA6009EF64FC6004EFB4FB15
:103F3F00030224AE9006C1E0C394F750509006C11F
:103F4F008046900265E07002A3E060419006C1E0F8
:103F5F00FF900269E02FF0900267E475F0011223E1
:103F6F00A9FC746C25F0F58274023CF583EFF09098
:103F7F00026574FFF5F012239345F0701090026301
:0E3F8F00E0FF1224AE90026AE0FF1240FE2214
:043498004103CC0020
:1034CC00E49006ADF0A37403F0E4A3F0124EE87E92
:1034DC00E07F017B017A0679AE90065AE4F0A304F2
:1034EC00F01244B87E007F467D007B017A03794060
:1034FC00122462E49006ADF09006ADE0FFC3940E8A
:10350C004003023592EFC39408EF75F0055050A4B8
:10351C002440F582E43403F58374FFF0EF75F00575
:10352C00A42443F582E43403F5837432F0EF75F090
:10353C0005A42442F582E43403F583E4F0EF75F03E
:10354C0005A42441F582E43403F583E4F0EF75F02F
:10355C0005A42444F582E43403F583E4F0800DA43F
:10356C002440F582E43403F58374FFF0EF75F00525
:10357C00A42443F582E43403F5837432F09006AD51
:10358C00E004F0023504E49006ADF09006ADE0FFE7
:10359C00C3941E502A75F046EFA42402F582E5F080
:1035AC0034E0AF82FE7B017A03794090065AE4F056
:1035BC00A37446F01244B89006ADE004F080CC7EC3
:1035CC00E07F007B017A0679AF90065AE4F0A30401
:0735DC00F01244B80249ACF3
:064F2E00E49003CCF02228
:074F0F009003CC7401F022B5
:104DA90020191030150D9003CCE07007AF1F124B7E
:044DB90032D21922B7
:104CFC0090E000E493F46007A3E493640360031270
:084D0C0034CCE4F561C2192268
:10493700E561C3941E501FE56175F046A42402F992
:1049470074E035F0FA7BFF78407C037D017E007FC1
:0749570046122246C219229C
:10482A00E561C3941E5029124EE875F046E561A46D
:10483A002402F582E5F034E0AF82FE7B017A037947
:10484A004090065AE4F0A37446F01244B81249ACF8
:01485A00223B
:0B4EAD00121A1B12482AC219024CCB3B
:0539C6009005DEEDF0AC
:1039CB009005E0E004F09005E3EFF0A3EBF0900539
:1039DB00DEE0FF9005E3E0FED39F4003023A7975EA
:1039EB00F046EEA42402F582E5F034E0AF829005B8
:1039FB00E5F0A3EFF09005E4E075F046A42402F5A2
:103A0B0082E5F034E0AF829005E7F0A3EFF0E490AD
:103A1B0005E1F0A3F09005E7E475F0011223A9AFDF
:103A2B00F0FE9005E5E0FCA3E0F5828C83E493FDCA
:103A3B00123D919005E6E004F070069005E5E00478
:103A4B00F09005E2E004F070069005E1E004F0C3AD
:103A5B009005E2E094469005E1E0940040B71249EE
:0E3A6B00AC9005E3E004F0A3E004F00239D9CA
:013A7900222A
:052BEB00900624EDF04E
:102BF000900629EFF0A3EBF0900624E0FF90062961
:102C0000E0D39F4003022D5CA3E075F046A42402AC
:102C1000F582E5F034E0AF82900625F0A3EFF0E412
:102C200090062BF0A3F090062BE0FEA3E0FFC394E8
:102C300046EE94005038900625E0FCA3E0F5828C27
:102C400083E493FD74862FF582E43403F583EDF07D
:102C5000900626E004F07006900625E004F0900649
:102C60002CE004F070C090062BE004F080B89006D1
:102C700029E075F046A42402F582E5F034E0AF8245
:102C8000900627F0A3EFF090062AE075F046A42402
:102C900002F582E5F034E0AF82900625F0A3EFF074
:102CA000E490062BF0A3F0900625E475F0011223C2
:102CB000A9AFF0FE900627E0FCA3E0F5828C83E448
:102CC00093FD123D91900628E004F07006900627CF
:102CD000E004F090062CE004F0700690062BE0046F
:102CE000F0C390062CE0944690062BE0940040B789
:102CF000900629E075F046A42402F582E5F034E060
:102D0000AF82900627F0A3EFF0E490062BF0A3F03B
:102D100090062BE0FCA3E0FDC39446EC9400502CFD
:102D2000900627E475F0011223A9AFF0FE74862DFA
:102D3000F582E43403F583E0FD123D9190062CE02A
:102D400004F070CC90062BE004F080C41249AC90E3
:0C2D50000629E004F0A3E004F0022BF8D8
:012D5C002254
:0B3A7A00900608EFF0A3EDF0A3EBF0C6
:103A8500A2AFE433A3F0C2AF124F08900609E0FEDF
:103A9500900608E0FDEDFF900610EEF0A3EFF0E4D0
:103AA50090060CF090060AE0FF900610E0FCA3E0FB
:103AB500FD7B017A03798690063CE4F0A37446F019
:103AC500124AAA900611E02446F0900610E0340050
:103AD500F090060CE075F046A42402F974E035F088
:103AE500FAA374FFF0A3EAF0A3E9F0124EE89006FA
:103AF5000DA3E0FAA3E0AE02FF7B017A037986907D
:103B0500065AE4F0A37446F01244B81249AC900684
:103B15000CE004F0E0C3941E408AAF1F124E4090A3
:073B2500060BE024FF92AF44
:013B2C002276
:0B3CFE0090062DEFF0A3EDF0A3EBF01B
:103D0900A2AFE433A3F0C2AF124F0890062EE0FE33
:103D190090062DE0FDEDFF900632EEF0A3EFF0E402
:103D2900900631F0900631E0FFC3941E504C75F0B7
:103D390046EFA42402F582E5F034E0AF82FE900656
:103D490034F0FAA3EFF0FB90062FE0FF900632E083
:103D5900FCA3E0FDA9037BFF900644E4F0A37446AD
:103D6900F0124C98900633E02446F0900632E03485
:103D790000F0900631E004F080AAAF1F124E409087
:073D89000630E024FF92AFB9
:013D90002210
:0D4E5A007E057F7A8E5A8F5B8E588F59220D
:084F0000759810D2ACC2BC226E
:064F3400124E5A024F006C
:014F48002246
:104DD000E559655B7004E558655A60037F01227FE1
:024DE0000022AF
:104AEE00055BE55BAE5A7002055A14F5828E83E0C3
:104AFE00FF7498B55B0B7405B55A06755A05755B50
:014B0E007A2C
:014B0F002283
:031A0F000244711D
:10447100C0E0C083C082C0D030982EC298855982D6
:10448100855883E599F00559E55970020558B498A6
:104491000BE558B4050675580575597AE559B55BAC
:1044A10008E558B55A03124F48309902C299D0D045
:0744B100D082D083D0E0327D
:10328B00205072696D6F2056657273696F6E2020C6
:10329B00200020496E697469616C697A696E6720D8
:1032AB00202020004D6F6E6F00506F6C7900205006
:1032BB00570041667400253364006275733A2563C9
:1032CB002043683A25326420257300547225632508
:1032DB0032642046743A416E20566C3A2563005492
:1032EB0072256325326420257325326420566C3A8F
:1032FB0025630046740046743A0058706F73653A44
:10330B00252B3364202056656C3A25630042757378
:10331B003A2563204368616E3A436C6F636B0044DC
:10332B0069763A2025642F252D3264203A202564B6
:10333B002F252D3264004275733A25632043686153
:10334B006E6E656C3A25326400436E74726C6C72EF
:10335B00733A00000AFF432E000CFF472A0104FFBB
:10336B004229010AFF485B010FFF490F000AFF4387
:10337B002E000CFF472A0108FF4229010FFF490FBE
:10338B00000FFF4381010BFF4C48010FFF4C630003
:10339B000FFF43810105FF47C60107FF4681010C63
:0833AB00FF47F8010EFF46BACE
:10349C00C1150F3441424344454647484A4B4C4DB5
:1034AC004E50000643FF32AFFF32B40624FF32B950
:0F34BC00FF32BD0A2A0102030406080C10182073
:1048E300E4900552F0900551F0900550F090054F7B
:1048F300F090054EF090067274FFF0A37432F0A3AB
:0C490300749DF07BFF7A32798B0246F342
:064F3A00E4900530F022B6
:103C69009006B8EEF0A3EFF0AF051DEF7003023C2C
:103C7900FD9006B8E0FEA3E0F5828E83A3A3E4934A
:103C8900FB740193FA740293F9900530E0FF75F023
:103C990005A42436F582E43405F583EBF0A3EAF0B4
:103CA900A3E9F09006B8E0FAA3E0FBF5828A83E481
:103CB90093FEEF75F005A42434F582E43405F58309
:103CC900EEF08B828A83740193FF900530E075F0E2
:103CD90005A42435F582E43405F583EFF090053029
:103CE900E004F09006B9E02405F09006B8E034004D
:053CF900F0023C712205
:1041CA00900553E0FBA3E0FAA3E0F912226CFE7516
:1041DA00F005A42434F582E43405F583E0FFEE7596
:1041EA00F005A42435F582E43405F583E0FD124E8A
:1041FA007F900553E0FBA3E0FAA3E0F912226C7565
:10420A00F005A42436F582E43405F583E0F9A3E049
:0F421A00FAA3E0900531C9F0A3EAF0A3E9F0227E
:10495E00900553E0FBA3E0FAA3E0F912226C700776
:10496E00900530E01222D4900553E0FBA3E0FAA3A9
:07497E00E0F974FF0222B210
:104BB500900553E0FBA3E0FAA3E0F974011222B2D9
:104BC50012226CFF900530E0B50704E41222D422CE
:0D19D50035F0FA7B01E0FD7482900684F08D
:1019E200ED1222B212226CFF3395E0FE900684E0E3
:1019F200FDD3EF9D7480F86E984003E0800B1222B5
:0D1A02006CC3648094805004E41222D4224E
:0B4B1000F583E0C4540FFFAD067B07E7
:104B1B009006C2EFF0AF037B017A0679C2EF121950
:074B2B00DE9006C2E0FF224C
:10432E0090054EE0FE75F005A42440F582E43403BA
:10433E00F583E02FF0EE75F005A42440F582E43409
:10434E0003F583E0FFB4FE13EE75F005A42440F5EB
:10435E0082E43403F583740FF08015EFB41011EE80
:10436E0075F005A42440F582E43403F58374FFF060
:03437E00024DA944
:1043810090054EE0FE75F005A42440F582E4340367
:10439100F583E02FF0EE75F005A42440F582E434B6
:1043A10003F583E0FFB4FE13EE75F005A42440F598
:1043B10082E43403F5837410F08015EFB41111EE2B
:1043C10075F005A42440F582E43403F58374FFF00D
:0343D100024DA9F1
:10472A009006C3EFF090054EE075F005A42441F918
:10473A00740335F0FA7B019006C3E0FD90054EE064
:10474A00C3940450047F0280027F01900684EFF034
:06475A001219E2024DA954
:1042290090054EE0FE75F005A42444F582E43403BC
:10423900F583E02FF0EE75F005A42444F582E4340B
:1042490003F583E0FFD3648094B04013EE75F00565
:10425900A42444F582E43403F5837430F08019C34F
:10426900EF648094505011EE75F005A42444F58252
:0B427900E43403F58374D0F0024DA97B
:10485B009006C4EFF090054EE075F005A42443F9E3
:10486B00740335F0FA7B019006C4E0FD9006847466
:10487B0063F01219E2124DA990054EE0FF0244FEBF
:10490F009006C5EFF090054EE075F005A42442F92E
:10491F00740335F0FA7B019006C5E0FD90068474B0
:08492F0009F01219E2024DA982
:1047C600AE0790054EE075F005A42441F582E43469
:1047D60003124B10EF540FC454F0FF90054EE075D2
:1047E600F005A42441F582E43403F583E0540F4F29
:0247F600F022AF
:10468100AE0790054EE075F005A42441F582E434AF
:1046910003F583E0540FFFAD067B09124B1BEF546A
:1046A1000FFF90054EE075F005A42441F582E43436
:0946B10003F583E054F04FF02200
:1047F800AE0790054EE075F005A42442F582E43436
:1048080003124B10EF540FC454F0FF90054EE0759F
:10481800F005A42442F582E43403F583E0540F4FF5
:02482800F0227C
:1046BA00AE0790054EE075F005A42442F582E43475
:1046CA0003F583E0540FFFAD067B09124B1BEF5431
:1046DA000FFF90054EE075F005A42442F582E434FC
:0946EA0003F583E054F04FF022C7
:104C48009006C6EFF090054EE075F005A42441F9F2
:0B4C580074039006C61219D5024DA986
:104C63009006C7EFF090054EE075F005A42442F9D5
:0B4C730074039006C71219D5024DA96A
:10408F0090069DEBF0A3EAF0A3E9F0A3EDF0C39443
:10409F0002502EE075F003A42424F8860308E6FAF4
:1040AF0008E6F9C003C00290069DE0FBA3E0FAA367
:1040BF00E0F8AC02AD03D002D0037E007F030222F2
:1040CF004690050B74FFF0A37432F0A374C1F09007
:1040DF0006A0E024FEFEE434FF90050EF0A3CEF020
:0F40EF0090069DE0FBA3E0FAA3E0F9121E7622F3
:101A2700124F3A90054EE0FFC394084003021C7B17
:101A3700EF75F005A42442F582E43403F583E0FF53
:101A47007D0112428490050B74FFF0A37432F0A35A
:101A570074C5F090054EE0FF2434F8E690050EF0CB
:101A6700EF75F005A42440F582E43403F583E02400
:101A770001FF90050FE4F0A3EFF090054EE075F03D
:101A870005A42441F582E43403F583E075F003A44B
:101A97002443F8860308E6FA08E6F9900511EBF007
:101AA700A3EAF0A3E9F07B017A057956121E769036
:101AB700054EE0FFC394044003021C2AEF75F005AE
:101AC700A42444F582E43403F583E07D0230E7047F
:091AD7007F0B80027F0A12428499
:101AE00090054EE0FF75F005A42443F582E434032D
:101AF000F583E0FD7C00900578ECF0A3EDF0643216
:101B0000705190050B74FFF0A37432F0A374D6F0FB
:101B1000A37402F0EF75F005A42444F582E43403C5
:101B2000F583E0FF5480FD3395E04D6006EFF4044B
:101B3000FF801390054EE075F005A42444F582E47F
:101B40003403F583E0FFEF3395E090050FF0A3EF4A
:101B5000021C03900578E0FEA3E0FFD39432EE640C
:101B60008094804005E024CE8011C3EF9432EE646F
:101B7000809480500E900579E024CFF0900578E0B5
:101B800034FFF090050B74FFF0A37432F0A374EAF5
:101B9000F0A37402F090054EE075F005A42444F51E
:101BA00082E43403F583E0FF5480FD3395E04D601B
:101BB00006EFF404FF801390054EE075F005A424B1
:101BC00044F582E43403F583E0FFEF3395E09005BC
:101BD0000FF0A3EFF0900578E0FEA3E0FFC394F7C9
:101BE000EE6480947F7BFF50067A3279FE80047A1F
:101BF000337901900511EBF0A3EAF0A3E9F0A3EE2D
:101C0000F0A3EFF0A37401F0FB7A057967121E765A
:101C10007E337F5E7D05123C699005537401F0A30D
:101C20007405F0A3744FF0021DF790050B74FFF0DC
:101C3000A37433F0A37405F090054EE075F005A48D
:101C40002444F582E43403F583E0FE3395E0900507
:101C50000EF0A3CEF0A37401F0FB7A057967121E93
:101C6000767E337F777D04123C699005537401F0D2
:101C7000A37405F0A37450F0021DF790054EE075B3
:101C8000F005A42440F582E43403F583E02401FF49
:101C9000EF641190050B6003021D4E74FFF0A374F6
:101CA00033F0A37418F090054EE02434F8E6900564
:101CB0000EF07B017A057956121E7690050B74FFA3
:101CC000F0A37433F0A3742AF090054EE0FF75F092
:101CD00005A42441F582E43403F583E0FEC4540FE7
:101CE0002401FCE43390050EF0A3CCF0EE540F2455
:101CF0002AF8E6FC3395E0A3F0A3CCF0EF75F005ED
:101D0000A42442F582E43403F583E0FFC4540F2495
:101D100001FCE433900512F0A3CCF0EF540F242A19
:101D2000F8E6FE3395E0A3F0A3CEF07B017A0579C7
:101D300067121E767E337F9A7D05123C69900553AB
:101D40007401F0A37405F0A37452F0021DF774FF40
:101D5000F0A37433F0A37441F090054EE0FF2434F7
:101D6000F8E690050EF0EF75F005A42440F582E446
:101D70003403F583E02401FFE43390050FE4F0A37E
:101D8000EFF07B017A057956121E7690050B74FFF1
:101D9000F0A37433F0A37454F07B017A05796712D1
:101DA0001E7690054EE075F005A42441F582E434DA
:101DB00003F583E0FD7B017A05797012408F900571
:101DC0004EE075F005A42442F582E43403F583E087
:101DD000FD7B017A05797412408F900573743AF097
:101DE0007E337F8B7D03123C699005537401F0A311
:101DF0007405F0A37451F09006727401F0A3740599
:101E0000F0A37467F07B017A0579561246F302411C
:011E1000CA07
:03000000020A00F1
:03000300021A03DB
:03000B00021A06D0
:03001300021A09C5
:03001B00021A0CBA
:03002300021A0FAF
:03002B00021A12A4
:03003300021A1599
:03003B00021A188E
:03004300021A1B83
:03004B00021A1E78
:03005300021A216D
:03005B00021A2462
:03006300021A2757
:03006B00021A2A4C
:03007300021A2D41
:100A0000E4F5D9E5EF7480F5FF7402F5EF787FE443
:100A1000F6D8FD9000007F007E10E4F0A3DFFCDE3E
:070A2000FA758161020A6210
:100A2700021626E493A3F8E493A34003F68001F2A9
:100A370008DFF48029E493A3F85407240CC8C333D0
:100A4700C4540F4420C8834004F456800146F6DF9F
:100A5700E4800B01020408102040809033B3E47E49
:100A6700019360BCA3FF543F30E509541FFEE49394
:100A7700A360010ECF54C025E060A840B8E493A35B
:100A8700FAE493A3F8E493A3C8C582C8CAC583CA86
:100A9700F0A3C8C582C8CAC583CADFE9DEE780BE3E
:0134CB000000
:10217600E709F608DFFA8046E709F208DFFA803E4B
:1021860088828C83E709F0A3DFFA8032E309F60838
:10219600DFFA8078E309F208DFFA807088828C83A0
:1021A600E309F0A3DFFA806489828A83E0A3F60854
:1021B600DFFA805889828A83E0A3F208DFFA804C2E
:1021C60080D280FA80C680D4806980F28033801005
:1021D60080A680EA809A80A880DA80E280CA80336E
:1021E60089828A83ECFAE493A3C8C582C8CCC583E6
:1021F600CCF0A3C8C582C8CCC583CCDFE9DEE780B6
:102206000D89828A83E493A3F608DFF9ECFAA9F034
:10221600EDFB2289828A83ECFAE0A3C8C582C8CC8A
:10222600C583CCF0A3C8C582C8CCC583CCDFEADEA3
:10223600E880DB89828A83E493A3F208DFF980CC05
:1022460088F0EF60010E4E60C388F0ED2402B404FE
:102256000050B9F582EB2402B4040050AF232345A5
:0622660082239021C673E3
:10226C00BB010689828A83E0225002E722BBFE0270
:09227C00E32289828A83E49322A3
:10228500BB010CE58229F582E5833AF583E022500E
:1022950006E92582F8E622BBFE06E92582F8E22258
:0D22A500E58229F582E5833AF583E4932272
:1022B200BB010989828A83F8E028F022500327F7BC
:1022C20022BBFE05F8E328F3228A838982F8E4938D
:0222D2002822C0
:1022D400BB010689828A83F0225002F722BBFE01E9
:0222E400F322E3
:1022E600F8BB010DE58229F582E5833AF583E8F02E
:1022F600225006E92582C8F622BBFE05E92582C8DA
:02230600F222C1
:10230800BC000BBE0029EF8DF084FFADF022E4CCB9
:10231800F875F008EF2FFFEE33FEEC33FCEE9DEC82
:10232800984005FCEE9DFE0FD5F0E9E4CEFD22EDC8
:10233800F8F5F0EE8420D21CFEADF075F008EF2F12
:10234800FFED33FD4007985006D5F0F222C398FD03
:052358000FD5F0EA22A0
:10235D00C2D5EC30E709B2D5E4C39DFDE49CFCEE9B
:10236D0030E715B2D5E4C39FFFE49EFE122308C3E8
:10237D00E49DFDE49CFC800312230830D507C3E4E3
:06238D009FFFE49EFE220A
:10239300C5F0F8A3E028F0C5F0F8E58215827002D5
:0623A3001583E038F02272
:1023A900A3F8E0C5F025F0F0E582158270021583E7
:0623B900E0C838F0E82244
:1023BF00EB9FF5F0EA9E42F0E99D42F0E89C45F074
:0123CF0022EB
:1023D0007401FF3395E0FEFDFCA3A3A3E0CF2FF033
:1023E000E582158270021583E0CE3EF0E58215820B
:1023F00070021583E0CD3DF0E582158270021583F1
:05240000E0CC3CF022DD
:10240500A8828583F0D083D08212241C12241C124A
:10241500241C12241CE473E493A3C583C5F0C5836F
:10242500C8C582C8F0A3C583C5F0C583C8C582C821
:012435002284
:10243600D083D082F8E4937012740193700DA3A335
:1024460093F8740193F5828883E473740293686049
:06245600EFA3A3A380DF49
:06245C008A838982E4730B
:101E1100E51A240BF582E43405F583E0051A2290D6
:101E2100050830070390050BE475F00112248E02BA
:101E3100226C2000E97F2ED2008018EF540F2490ED
:101E4100D43440D4FF30040BEF24BFB41A00500344
:101E51002461FFE51B6002151B051EE51E700205CE
:101E61001D30070E900508E475F00112248EEF0273
:101E710022D40249857403D2078003E4C207F51A0C
:101E81009005081224A5E4F51BF51DF51EE51B6060
:101E9100077F20121E5480F5751CFFC201C200C2CB
:101EA10002C203C205C206C208121E20FF700D3015
:101EB10007057F00121E65AF1EAE1D22B4255FC24D
:101EC100D5C204121E20FF24D0B40A00501A75F0A6
:101ED1000A781B30D50508B6FF0106C6A426F620F0
:101EE100D5047002D20380D924CFB41A00EF500474
:101EF100C2E5D204022066D20180C6D20080C0D2DF
:101F01000280BCD2D580BAD20580B47F20121E5483
:101F11002002077401B51B0040F1121E11FF121EB1
:101F210054021E8ED208D2068095121E11FB121E7B
:101F310011FA121E11F94A4B700679377A217BFF8B
:101F410020022EE51B602A7E008E827583001222FC
:101F51008560060EEE651C70F0C2D5EBC0E0EAC0EC
:101F6100E0E9C0E0EE1220ADD0E0F9D0E0FAD0E037
:101F7100FB12226CFF60AAEBC0E0EAC0E0E9C0E01E
:101F8100121E54D0E02401F9D0E03400FAD0E0FB75
:101F9100E51C0460DCD51CD980877BFF7A2079A9F8
:101FA100D202809C791080027908C206C20880089A
:101FB100D2D5790A8004790AC2D5E51C047002F5EC
:101FC1001CE4FAFDFEFF121E11FC7B082001131216
:101FD1001E11FD7B1030000A121E11FE121E11FF90
:101FE1007B20EC3382D592D55013C3E43000069F99
:101FF100FFE49EFEE42001039DFDE49CFCE4CBF89C
:10200100C201EC700CCFCECDCCE824F8F870F3808F
:1020110017C3EF33FFEE33FEED33FDEC33FCEB334F
:10202100FB994002FB0FD8E9EB300105F8D0E0C481
:1020310048B201C0E00AEC4D4E4F78207B0070C2DF
:10204100EAB51C0040BCC0E01220AFD0F0D0E020C7
:102051000104C4C0E0C4B201C0F0121E3DD0F0D5ED
:10206100F0EB021E8E1224361F2B531FA5581EFCA7
:102071004C1EF8421FA94F1FB1441FB1491F114304
:082081001FB7551F9B461F9B72
:10208900451F9B472157501F002D1F042E1F272B2B
:102099001F08231F252021402A1EC04800001F1F9A
:1020A9003F3F3F00790AA2D5200314300509B91032
:1020B900020404B9080104A2D52006025001042033
:1020C90002689202B51B005034C0E07F203003192A
:1020D9007F30A20272067205500F122106C202C297
:1020E90006C205C2087F30800F300503E9C0E0123F
:1020F9001E54300503D0E0F9D0E0B51BCC300517EC
:102109007F30B9100C121E547F583004077F788035
:1021190003B90803121E543002057F2D021E547F95
:10212900202008F87F2B2006F322920280CF286E08
:10213900756C6C2900D201121E113001F8C20178A8
:102149001B30D50108F6021EC02D50434958121EF6
:10215900112403B405004001E490215293121E4555
:0D216900743A121E45D203751B04021FA517
:10246200EF4E6012EF60010EEDBB010B89828A8391
:10247200F0A3DFFCDEFA2289F05007F709DFFCA99E
:0C248200F022BBFEFCF309DFFCA9F022F5
:10248E00F8E0FBA3A3E0F925F0F0E58215827002D7
:07249E001583E0FA38F0227B
:0924A500EBF0A3EAF0A3E9F02238
:10498500EFB40A07740D124990740A309811A8996A
:10499500B8130CC2983098FDA899C298B811F63092
:0749A50099FDC299F599226A
:00000001FF
